S024000062696E2F6F70656E626C745F6F6C696D65785F73746D3332683130332E73726563A3
S3150800000000500020B5010008FB010008FD010008AA
S31508000010FF010008010200080302000800000000B2
S3150800002000000000000000000000000005020008B3
S315080000300702000800000000090200080B02000879
S315080000400F02000811020008130200081502000832
S3150800005017020008190200081B0200081D02000802
S315080000601F020008210200082302000825020008D2
S3150800007027020008290200082B0200082D020008A2
S315080000802F02000831020008330200083502000872
S3150800009037020008390200083B0200083D02000842
S315080000A03F02000841020008430200084502000812
S315080000B047020008490200084B0200084D020008E2
S315080000C04F020008510200085302000855020008B2
S315080000D057020008590200085B0200085D02000882
S315080000E05F020008610200086302000808B540F2D2
S315080000F0F800074BC2F200001B1A062B00D808BDF1
S3150800010040F20003C0F20003002BF8D09847F6E748
S31508000110FB00002008B540F2F80040F2F803C2F2EE
S315080001200000C2F200031B1A9B1003EBD37359108D
S3150800013000D108BD40F20002C0F20002002AF8D041
S315080001409047F6E710B540F2F804C2F200042378A7
S3150800015073B9FFF7CBFF40F20003C0F200032BB1DF
S3150800016042F66020C0F60000AFF30080012323703A
S3150800017010BD00BF08B540F20003C0F200034BB142
S3150800018042F6602040F2FC01C0F60000C2F200010F
S31508000190AFF3008040F2F800C2F2000003682BB10A
S315080001A040F20003C0F2000303B19847BDE80840D7
S315080001B0B0E700BF06498D460649074A074B9A42EB
S315080001C0BEBF51F8040B42F8040BF8E70448004791
S315080001D000500020642A000800000020F8000020D3
S315080001E0E50100081F49204A002301E041F8043BC5
S315080001F09142FBD301F0C8F9FEE7FEE7FEE7FEE70A
S31508000200FEE7FEE7FEE7FEE7FEE7FEE7FEE7FEE7B8
S31508000210FEE7FEE7FEE7FEE7FEE7FEE7FEE7FEE7A8
S31508000220FEE7FEE7FEE7FEE7FEE7FEE7FEE7FEE798
S31508000230FEE7FEE7FEE7FEE7FEE7FEE7FEE7FEE788
S31508000240FEE7FEE7FEE7FEE7FEE7FEE7FEE7FEE778
S31508000250FEE7FEE7FEE7FEE7FEE7FEE7FEE7FEE768
S31508000260FEE7FEE7F80000207807002040F21413A6
S31508000270C2F200031B78CBB94FF48053C4F20203D1
S315080002809A6942F010029A614FF48053C4F201034E
S315080002905A6822F470425A605A6842F4E0425A6038
S315080002A040F21413C2F2000301221A7001284FF417
S315080002B08053C4F201034FF400620CBF5A611A61FD
S315080002C0704700BF4FF40063C4F20103986800F05A
S315080002D00100704708B538B940F26C73C2F20003E2
S315080002E01B6801221A8208BD40F26873C2F2000335
S315080002F01B681B68984740F26C73C2F200031868C3
S315080003000A3008BD08B538B940F26C73C2F200036A
S315080003101B6801221A8208BD40F26873C2F2000304
S315080003201B689B68984740F26C73C2F20003186812
S315080003300C3008BD08B538B940F26C73C2F2000338
S315080003401B6802221A8208BD40F23C73C2F20003FF
S3150800035000221A8040F26C73C2F200031A681378FE
S3150800036013F07F0317D1537A13F0200F1FBF40F203
S315080003703C72C2F200020221117013F0400F40F2E3
S315080003803C73C2F200031A7814BF42F0010222F04D
S3150800039001021A702BE0012B35D0022B38D1537984
S315080003A003F00F0213F0800F10D0920002F1804282
S315080003B002F5B842136803F03003102B17D140F248
S315080003C03C73C2F2000301221A7010E0920002F197
S315080003D0804202F5B842136803F44053B3F5805FD0
S315080003E001BF40F23C73C2F2000301221A7040F2C8
S315080003F06873C2F200031B681B69984740F23C7099
S31508000400C2F2000008BD40F23C70C2F2000008BD0E
S31508000410002008BDF8B540F26C73C2F200031C68F0
S31508000420238A227A002B08BF042A29D140F2151301
S31508000430C2F200031B78012B1AD145F65043C4F2C9
S3150800044000031A6892B243F20203C2F2000313448D
S315080004505B0000221A6040F27473C2F20003302176
S31508000460198040F21513C2F200031A70042633E00D
S3150800047040F27473C2F2000310221A8007262BE09A
S31508000480A58AAB4294BF042602269D4228BF1D4674
S31508000490A369ADB2284698470746002000F030FF0A
S315080004A0014638462A4600F035FE0020294600F067
S315080004B047FF238A5B1B2382638A1D44658240F2B9
S315080004C07473C2F2000330221A8040F27273C2F2C9
S315080004D000034FF440521A8040F26C73C2F20003D4
S315080004E01B681E72F8BD00BF10B582B040F26C736F
S315080004F0C2F200031A685378062B25D1137813F035
S315080005007F0F18BF002340F0BA809378012B06D1DD
S3150800051040F24473C2F200031B68DB69AFE0022BAA
S3150800052006D140F24473C2F200031B681B6AA6E0B8
S31508000530032B18BF002340F0A28040F24473C2F296
S3150800054000031B685B6A9AE0002B5AD15188002980
S3150800055057D1516821F47F41B1F5003F51D1137845
S3150800056013F07F0302D1918800297FD0012B19D17E
S3150800057040F24473C2F200031B689B69507900215C
S315080005809847002300287AD140F26C73C2F2000320
S315080005901B689A7A40F23533C0F60003002A08BF72
S315080005A000236CE0022B18BF002368D1537903F0AF
S315080005B00F0203F0700113F0800F4FEA820303F174
S315080005C0804303F5B843186814BF00F0300000F400
S315080005D0405040F2E803C2F200031B78934298BFEA
S315080005E000234CD9D1F1010138BF0021002808BFEA
S315080005F0002140F23533C0F60003002908BF002366
S315080006003DE0082B0AD1127802F07F0240F2D5238A
S31508000610C0F60003002A18BF002330E00A2B18BFD3
S3150800062000232CD1137803F07F03012B18BF002376
S3150800063025D1937AFBB15388FBB9536823F47F43DA
S31508000640B3F5803F18BF002319D140F24473C2F2B4
S3150800065000031B689B6950790021984740F20533CF
S31508000660C0F60003002818BF002308E040F235331F
S31508000670C0F6000303E0002301E00023FFE75BB1B7
S3150800068040F26C72C2F2000212680024548293612E
S3150800069020469847204616E040F24473C2F200030B
S315080006A01B681A6940F26C73C2F200031B6858781B
S315080006B09047032807D140F26C73C2F200031B6807
S315080006C009221A724FE040F26C73C2F200031B68EB
S315080006D01A8A4FF6FF718A4204BF09221A7242D05B
S315080006E0022800D012B908221A723CE093F90010C9
S315080006F000292FDAD98801910198824202D9019AF4
S315080007001A821CE08A421AD240F24471C2F20001EF
S31508000710096891F82C108A4206D240F21512C2F2E4
S315080007200002002111700AE092FBF1F001FB102291
S315080007302AB940F21512C2F200020121117040F2E4
S315080007404472C2F20002126892F82C209A82FFF7CD
S3150800075061FE08E003221A7240F27273C2F20003C5
S315080007604FF440521A8002B010BD00BF70B540F277
S315080007706C73C2F200031C68218AA369B3B1A9B1DC
S31508000780A58A8D4228BF0D46ADB22846984706462B
S31508000790238A5B1B2382638A2B446382002000F032
S315080007A0BFFD014630462A4600F0CAFC238A83B1BB
S315080007B040F27273C2F200034FF440521A800020CE
S315080007C0014600F0BDFD40F27473C2F20003302208
S315080007D01A80238AA28A934207D340F26C73C2F224
S315080007E000031B6803221A7270BD3BB140F26C739A
S315080007F0C2F200031B6805221A7270BDD3B940F213
S315080008006C73C2F200031B6806221A7245F650433F
S31508000810C4F200031A6892B243F20203C2F200035A
S3150800082013445B0000221A6040F27473C2F200039C
S3150800083030221A8070BD00BF08B540F26C73C2F250
S3150800084000031A68D17840F2E803C2F200035B7825
S3150800085099420DD893786BB993886BB9917240F227
S315080008606873C2F200031B685B689847002008BDDE
S31508000870022008BD022008BD022008BD10B540F2BE
S315080008804473C2F200031B689A6940F26C74C2F2A0
S31508000890000423685879D978904723689A7A9AB1D8
S315080008A0A0B91A79A2B99B78A3B9A8B940F2687316
S315080008B0C2F200031B68DB68984723685A79DA7224
S315080008C0DA781A73002010BD022010BD022010BD70
S315080008D0022010BD022010BD022010BD10B540F246
S315080008E06C73C2F200031A68137813F07F0305D1FC
S315080008F0537A23F020035372002010BD022B6FD1C8
S315080009005388002B6ED11379002B6DD1517921F0C4
S31508000910800011F0800F4FEA800303F1804303F54E
S31508000920B84319BF1C6804F030041B6803F440542C
S3150800093040F2E803C2F200031B78834256D9002C22
S3150800094056D0937A002B55D011F0800F12D0830021
S3150800095003F1804303F5B8431B6803F03003102BFB
S3150800096035D1C4B2204600F091FC2046302100F073
S315080009700DFC2CE0840004F1804404F5B844236897
S3150800098003F44053B3F5805F21D198B940F25C0374
S31508000990C2F2000393F82C1000F0E2FC22684BF632
S315080009A08F73134083F4405343F4004343F08003AA
S315080009B023600CE000F056FC22684BF68F73134058
S315080009C083F4405343F4004343F08003236040F22A
S315080009D06873C2F200031B685B699847002010BD64
S315080009E0022010BD022010BD022010BD022010BD3D
S315080009F0022010BD022010BD10B540F26C73C2F281
S31508000A0000031868427922F0800112F0800F4FEA3D
S31508000A10810303F1804303F5B84319BF1C6804F04A
S31508000A2030041B6803F4405440F2E803C2F20003A2
S31508000A301B78994227D243883BBB44B3837A43B396
S31508000A4012F0800F4FEA810202F1804202F5B842A5
S31508000A5011681DBF48F6BF730B4083F010034BF6B1
S31508000A608F7304BF0B4083F4805343F4004343F071
S31508000A708003136040F26873C2F200031B689B6927
S31508000A809847002010BD022010BD022010BD02208C
S31508000A9010BD022010BD00BF08B540F26C73C2F24B
S31508000AA000031B685A7A42F020025A7240F26873B1
S31508000AB0C2F200031B68DB699847002008BD00BF27
S31508000AC010B540F26C73C2F200031B685C781A78A2
S31508000AD012F07F0239D1092C02D1FFF7ADFE4DE0A5
S31508000AE0052C10D193F90320002AB8BF082270DB21
S31508000AF09A78002A67D19A88002A66D19B7A0020BC
S31508000B00002B3BD063E0032C0AD1DA78012A18BF00
S31508000B10022033D19B88022083BBFFF7BDFF2DE05F
S31508000B20012C18BF022029D1DA78012A18BF022021
S31508000B3024D19A8802200ABB5B7A13F0200F08BFDB
S31508000B4002201BD0FFF7CAFE18E0012A06D10B2C9B
S31508000B5018BF022012D1FFF791FE0FE0022A18BF34
S31508000B6002200BD1012C02D1FFF7B8FE06E0032CB8
S31508000B7018BF022002D1FFF73FFFFFE758B140F246
S31508000B804473C2F200031B685B6920469847032832
S31508000B9008BF09221DD00822D8B945F65043C4F229
S31508000BA000031A6892B243F20203C2F20003134426
S31508000BB05B0000221A6040F27473C2F2000330220E
S31508000BC01A80062205E0082203E0082201E008222E
S31508000BD0FFE740F26C73C2F200031B681A7210BD7D
S31508000BE040F26C73C2F200031B685A8A18B98988E6
S31508000BF08A1A1A82704708681044704708B540F286
S31508000C005C03C2F20003002093F82C1000F0A8FB46
S31508000C1040F26C73C2F200031B68187A08280CD1DC
S31508000C2040F27273C2F200034FF480521A8040F207
S31508000C307473C2F2000310221A80092814BF002018
S31508000C40012008BD70B545F65043C4F200031A6882
S31508000C5092B243F20403C2F2000313445B001A88FB
S31508000C60520002F1804202F5C04240F26C73C2F2B1
S31508000C7000031B68197A092919D0551C11781970AF
S31508000C8040F26C74C2F20004236852785A702668DF
S31508000C90B5F8030000F09CFB70802668B5F80700DD
S31508000CA000F096FBB0802368B5F80B20DA8040F296
S31508000CB06C73C2F200031B6801221A72DB8813B92F
S31508000CC0FFF7FEFE01E0FFF70FFCFFF797FF70BD89
S31508000CD008B540F26C73C2F200031B681B7A042B3A
S31508000CE018BF022B08BF082219D0052B18BF032BE3
S31508000CF008D1FFF73BFD40F26C73C2F200031B6894
S31508000D001A7A0CE0072B18BF082208D140F2447360
S31508000D10C2F200031B68DB6898470822FFE740F227
S31508000D206C73C2F200031B681A72FFF767FF08BDEF
S31508000D3070B440F2E803C2F200031D78002340F6BF
S31508000D400F760EE0DCB2A10001F1804101F5B84151
S31508000D500A68324042F4004242F0800222430A60A6
S31508000D600133AB42EED340F0800045F64C43C4F263
S31508000D700003186070BC704708B540F26C73C2F285
S31508000D8000031A68137A042B18BF022B08D1FFF741
S31508000D9041FB40F26C73C2F200031B681A7A1DE02D
S31508000DA0062B18BF082219D15378052B0DD11378B5
S31508000DB013F07F0F09D1D078FFF7BAFF40F26873B6
S31508000DC0C2F200031B681B6A984740F24473C2F2DA
S31508000DD000031B689B6898470822FFE740F26C737C
S31508000DE0C2F200031B681A72FFF708FF08BD00BFAE
S31508000DF0704700BF08B540F26C72C2F2000240F2BA
S31508000E004C73C2F20003136002221A7240F2447253
S31508000E10C2F2000240F25C03C2F20003136040F221
S31508000E206872C2F2000240F28C01C2F2000111603F
S31508000E301B68984708BD00BF2DE9F04383B000231F
S31508000E40ADF8063045F64447C4F2000740F276741A
S31508000E50C2F2000440F24876C2F2000640F21C08CC
S31508000E60C2F2000840F23809C2F2000940F272756F
S31508000E70C2F2000543E1238803F00F033370002B09
S31508000E8040F00F814FF4B843C4F200031A6892B2D7
S31508000E902A80298801F0300140F27472C2F20002F9
S31508000EA011802A8802F440522A8019684BF6BF72CC
S31508000EB00A4082F4005282F0200242F4004242F0D4
S31508000EC080021A60238803F010039BB2002B46D1D8
S31508000ED04FF4B844C4F20004226848F60F7313406E
S31508000EE02360FFF749FF22684BF6BF73134040F2B1
S31508000EF07272C2F20002128802F4805292B20AB1E9
S31508000F0083F4805340F27272C2F20002128802F42D
S31508000F10005292B20AB183F4005340F27472C2F2DC
S31508000F200002128802F0100292B20AB183F010038E
S31508000F3040F27472C2F20002128802F0200292B2E3
S31508000F400AB183F0200348F28002CFF6FF721A43F3
S31508000F5092B24FF4B843C4F200031A60D6E04FF4D5
S31508000F60B843C4F200031B689BB2ADF80630BDF85F
S31508000F70063003F400639BB2002B46D04FF4B84406
S31508000F80C4F20004226840F68F7313402360FFF70B
S31508000F9059FE22684BF6BF73134040F27272C2F2D2
S31508000FA00002128802F4805292B20AB183F4805386
S31508000FB040F27272C2F20002128802F4005292B231
S31508000FC00AB183F4005340F27472C2F20002128826
S31508000FD002F0100292B20AB183F0100340F2747262
S31508000FE0C2F20002128802F0200292B20AB183F01D
S31508000FF0200348F28002CFF6FF721A4392B24FF4EA
S31508001000B843C4F200031A6080E0BDF806301BB28C
S31508001010002B74DA4FF4B844C4F20004226840F690
S315080010208F7313402360FFF753FE22684BF6BF7396
S31508001030134040F27272C2F20002128802F4805221
S3150800104092B20AB183F4805340F27272C2F200027D
S31508001050128802F4005292B20AB183F4005340F2A5
S315080010607472C2F20002128802F0100292B20AB139
S3150800107083F0100340F27472C2F20002128802F082
S31508001080200292B20AB183F0200348F28002CFF61A
S31508001090FF721A4392B24FF4B843C4F200031A60BF
S315080010A034E09B0003F1804303F5B8431A6892B213
S315080010B0ADF80620BDF8062012B2002A09DA19682A
S315080010C040F68F720A401A603378013B59F823308C
S315080010D09847BDF8063003F080039BB27BB132789F
S315080010E0920002F1804202F5B842116848F60F7381
S315080010F00B4013603378013B58F8233098473B6818
S315080011009BB2238013F4004F7FF4B5AE03B0BDE85D
S31508001110F08300BF10B40132531001F1005101F5FC
S315080011204052520007E00178447841EA042122F847
S31508001130041B0230013B002BF5D15DF8044B7047C8
S315080011400132531001F1005101F54052520004E0FA
S31508001150116820F8021B013B0432002BF8D17047B6
S315080011604FF6F873034045F65042C4F20002136086
S31508001170704700BF800000F1804202F5B84210684F
S3150800118048F68F130340194311607047800000F139
S31508001190804202F5B842106848F6BF73034001F072
S315080011A0100080B208B183F0100301F0200189B263
S315080011B009B183F0200343F4004343F0800313602E
S315080011C0704700BF800000F1804202F5B8421068FF
S315080011D04BF68F73034001F4805080B208B183F454
S315080011E0805301F4005189B209B183F4005343F4E2
S315080011F0004343F080031360704700BF800000F18E
S31508001200804202F5B842116848F6BF730B4083F076
S31508001210300343F4004343F080031360704700BF74
S31508001220800000F1804202F5B84211684BF68F73D0
S315080012300B4083F4405343F4004343F080031360A8
S31508001240704700BF800000F1804202F5B84211687D
S3150800125040F60F630B4043F4004343F080031360EA
S31508001260704700BF800000F1804303F5B8431A6851
S3150800127012F4804F08D0196840F60F720A4042F4FB
S31508001280404242F080021A60704700BF800000F1B9
S31508001290804303F5B8431A6812F0400F08D019685E
S315080012A040F60F720A4042F4004242F0C0021A6049
S315080012B0704700BF45F65043C4F200031B689BB253
S315080012C003EBC00000F1005202F5405252004FF6FF
S315080012D0FE730B401360704745F65043C4F2000393
S315080012E01B689BB203EBC00043F20403C2F200037F
S315080012F003445B004FF6FE720A401A60704700BF4F
S3150800130045F65043C4F200031B689BB203EBC000CA
S3150800131000F1005303F540535B001888704700BF7F
S3150800132045F65043C4F200031B689BB203EBC000AA
S3150800133043F20403C2F2000303445B0018887047B3
S3150800134045F65043C4F200031B689BB203EBC0008A
S3150800135043F20203C2F2000303445B0019607047BC
S3150800136045F65043C4F200031B689BB203EBC0006A
S3150800137043F20603C2F2000303445B003E290BD97D
S315080013804A0911F01F0F04BF02F1FF3292B292020E
S3150800139042F400421A6070474A0811F0010F1CBF58
S315080013A0013292B292021A60704700BF45F6504366
S315080013B0C4F200031B689BB203EBC00043F20603AA
S315080013C0C2F2000303445B001888C0F309007047A3
S315080013D0C3B2000A40EA0320704700BF45F64443FB
S315080013E0C4F200030020186040F27073C2F20003D2
S315080013F04FF406421A8045F64043C4F200031A60C9
S31508001400704700BF70B50E4600F07F052846FFF707
S31508001410CDFF04462846FFF783FF0146304622469D
S31508001420FFF78EFE204670BD00B583B000230193FA
S3150800143000934FF48053C4F202031A6842F0010283
S315080014401A6059680022CFF6FF020A405A601A68E5
S3150800145022F0847222F480321A601A6822F48022FA
S315080014601A605A6822F4FE025A604FF41F029A6004
S315080014701A6842F480321A604FF48052C4F20202AB
S3150800148040F2DC51136803F400330093019B0133E7
S315080014900193009B13B9019B8B42F3D14FF4805300
S315080014A0C4F202031B6813F4003F06D142F6D800C3
S315080014B0C0F60000672100F0DBF94FF40053C4F2D0
S315080014C002031A6842F010021A601A6822F0030230
S315080014D01A601A6842F002021A604FF48053C4F286
S315080014E002035A685A605A6842F400525A605A68A7
S315080014F042F480625A605A6822F47C125A605A682A
S3150800150042F4E8125A601A6842F080721A604FF480
S315080015108052C4F20202136813F0007FFBD04FF426
S315080015208053C4F202035A6822F003025A605A68CA
S3150800153042F002025A604FF48052C4F20202536823
S3150800154003F00C03082BFAD14FF48053C4F20203BC
S315080015509A6942F004029A614FF40062C4F20102E9
S31508001560116821F00F011160116841F00401116042
S315080015705A6822F480025A60DA6942F40002DA6193
S3150800158003B05DF804FB00BF08B5FFF74DFF00F098
S31508001590A5F900F0B1F9FCE708B501F0FBF808BDBC
S315080015A008B501F03BF908BD08B540F21813C2F2B8
S315080015B000031B68052B01D101F0ECF808BD00BF3C
S315080015C008B545F64443C4F200031A6892B240F2DD
S315080015D07673C2F200031A801A8802F4007240F287
S315080015E07073C2F200031B881A4210D045F64443B2
S315080015F0C4F200034FF6FF521A6040F21613C2F205
S3150800160000031A780132D2B21A70FFF7CDFF40F202
S315080016107673C2F200031A8802F4004240F270732D
S31508001620C2F200031B881A4201D0FFF705FC40F2FC
S315080016307673C2F200031A8802F4806240F270736D
S31508001640C2F200031B881A420CD045F64443C4F282
S3150800165000034FF6FF321A6040F25C03C2F2000341
S315080016605B68984708BD00BF40F24C73C2F200039E
S315080016709B7A2BB140F21813C2F2000305221A60B6
S31508001680704700BF40F21813C2F2000304221A6022
S31508001690704700BF704700BF704700BF10B50628E7
S315080016A018BF002317D140F26C73C2F200031B68FF
S315080016B01A7802F07F02012A18BF00230BD15A7943
S315080016C042B99A7841F62D03C0F60003212A18BFBD
S315080016D0002300E000235BB140F26C72C2F2000204
S315080016E0126893610024548220469847204610BD0C
S315080016F0022010BD0220704721B9002814BF02201D
S31508001700002070470220704710B501F0B5F840F286
S315080017106C73C2F200031B6800249C7200F08EF8FA
S31508001720FFF75CFE40F21813C2F200031C6010BDFE
S3150800173010B540F26C73C2F200031B6800249C7259
S3150800174042F62012C0F60002D2795A72DC7220469E
S31508001750FFF706FD20464FF40071FFF70BFD204604
S315080017601021FFF713FD20464021FFF7B5FD20465F
S315080017708021FFF79FFD2046FFF764FD40F25C03DA
S31508001780C2F20003204693F82C10FFF7E9FD204625
S31508001790FFF746FD01202146FFF7ECFC01204FF438
S315080017A08071FFF787FD0120C021FFF795FD012015
S315080017B04021FFF7C5FD01204021FFF7D1FD01209B
S315080017C04FF44051FFF7FEFC01202021FFF7DEFC15
S315080017D02046FFF7ADFA40F21813C2F200030122C1
S315080017E01A6010BD08B540F2B801C2F20001FFF751
S315080017F0F7F908BD08B540F25401C2F20001FFF737
S31508001800EFF908BD08B540F26C73C2F200031B6815
S31508001810D978052908D840F2C003C2F2000303EBC1
S31508001820C101FFF7DDF908BD002008BD08B540F283
S31508001830B001C2F20001FFF7D3F908BD08B50120CF
S31508001840FEF714FD45F64043C4F2000301221A6070
S3150800185040F27072C2F200020020186045F6444158
S31508001860C4F2000108604FF4E0511180196008BD08
S3150800187008B500F0A9F8FCE708B500F09FF80128BC
S3150800188019D040F21C13C2F200031B78012B12D1A7
S3150800189000F0D0FD40F22013C2F200031B6803F5E6
S315080018A0FA63984207D340F21C13C2F200030022DF
S315080018B01A7000F0B1FA08BD08B540F21C13C2F25E
S315080018C0000301221A7000F0B5FD40F22013C2F29F
S315080018D000031860FFF7D0FF08BD00BF08B500F089
S315080018E097FA00F06FF800F07DFD00F055FD00F066
S315080018F00DF8FFF7E1FF08BD08B500F065F800F040
S3150800190087FD00F00FF8FFF7B7FF08BD08B500F030
S31508001910E3F900F08DFE40F2EC03C2F20003022266
S315080019201A7008BD08B540F22410C2F2000000F093
S31508001930DBFE01280BD140F2EC03C2F200030222BF
S315080019401A7040F22410C2F2000000F0E5F908BD52
S3150800195008B500F091FE08BD08B540F2EC03C2F2E6
S3150800196000031B78022B02D1C9B200F08BFE00F0EF
S31508001970CBF908BD40F2EC03C2F200031B78032B37
S3150800198005D8DFE803F0060602063F2070473F2029
S3150800199070470020704700BF40F2EC03C2F2000314
S315080019A01B78032B05D8DFE803F0060602063F205E
S315080019B070473F2070470020704700BF08B500F009
S315080019C099F908BD704700BF704700BF10B40023DF
S315080019D004E010F8011B0B44DBB221464C1E00291B
S315080019E0F7D1136001205DF8044B704740F2641389
S315080019F0C2F2000300225A70704700BF40F2641317
S31508001A00C2F20003FE22DA7018710222A3F84420FB
S31508001A10704700BF10B540F26414C2F200040023F8
S31508001A202370FFF7E3FFFF23E3700123A4F8443094
S31508001A3010BD00BF40F26413C2F20003FF22DA7041
S31508001A4000221A71597859719A71DA711A72062236
S31508001A50A3F84420704700BF08B50020FFF7CEFF63
S31508001A6008BD00BF40F26413C2F20003FF22DA7019
S31508001A7042F68812C0F600029A6400221A715A7158
S31508001A809A710721D9711A725A729A720822A3F8A2
S31508001A904420704740F26413C2F20003FF22DA7052
S31508001AA042689A640122A3F84420704710B540F2B0
S31508001AB06414C2F20004FF23E3704168A06CE21DBF
S31508001AC0FFF784FF207100236371A3710823A4F82C
S31508001AD0443010BD08B53120FFF790FF08BD00BFA0
S31508001AE038B540F26414C2F20004FF23E3700025FF
S31508001AF025716571FFF73EFFA071E5712572657264
S31508001B000723A4F8443038BD38B5FFF76FFF40F215
S31508001B106414C2F2000401252570FF23E370102324
S31508001B20237100236371FFF725FFA071FFF734FFC8
S31508001B30E071FFF731FFC0F3072020726572A572C6
S31508001B400823A4F8443000F027FC38BD38B505460C
S31508001B504478FFF70FFF0138844203DD2220FFF7A0
S31508001B604DFF38BD40F26414C2F20004201DA16C7A
S31508001B706A7800F06FF9FF23E3706A78A36C134460
S31508001B80A3646B780133A4F8443038BD38B50546EC
S31508001B904478FFF7EFFE0138844203DD2220FFF781
S31508001BA02DFF38BD696840F26414C2F20004A164CE
S31508001BB0201D6A7800F04EF9FF23E3706A78A36C5B
S31508001BC01344A3646B780133A4F8443038BD00BFCE
S31508001BD038B5044640F26413C2F200039D6CFFF761
S31508001BE0C9FE411E2846621C00F0DAFB18B93120EE
S31508001BF0FFF704FF38BD40F26414C2F20004FF2365
S31508001C00E370A56CFFF7B6FE2844451EA5640123BC
S31508001C10A4F8443038BD00BF38B504464578FFF708
S31508001C20A9FE0238854203DD2220FFF7E7FE38BD0C
S31508001C3040F26413C2F20003FF22DA700122A3F80D
S31508001C404420617831B900F0BBFBC0B93120FFF7F9
S31508001C50D5FE38BD40F26413C2F20003986CA21C8C
S31508001C6000F09EFB18B93120FFF7C8FE38BD617831
S31508001C7040F26413C2F200039A6C0A449A6438BDAF
S31508001C8008B540F26413C2F200034168986C00F08C
S31508001C908BFB18B93120FFF7B1FE08BD40F264137B
S31508001CA0C2F20003FF22DA700122A3F8442008BD1D
S31508001CB008B500F0B1F840F26413C2F20003FF223F
S31508001CC0DA700122A3F8442008BD00BF08B589B21E
S31508001CD0FFF742FE08BD00BF40F26413C2F20003DC
S31508001CE000221A709A6483F84220A3F844209A7056
S31508001CF05A70704740F26413C2F200031878003035
S31508001D0018BF0120704700BF40F26413C2F20003F7
S31508001D10002283F84220704708B50278FF2A02D1CC
S31508001D20FFF7F2FE53E040F26413C2F200031B7899
S31508001D30012B6BD1C93A352A46D8DFE802F033457C
S31508001D40454245453F363C39454545454545454562
S31508001D504545454545454545454545454545454525
S31508001D604545454545454545241E1B2145454527C9
S31508001D70452A2D30FFF7EAFE29E0FFF707FF26E0A0
S31508001D80FFF788FE23E0FFF791FE20E0FFF76AFEE3
S31508001D901DE0FFF761FE1AE0FFF74CFE17E0FFF7BC
S31508001DA039FE14E0FFF714FF11E0FFF735FF0EE0E8
S31508001DB0FFF796FE0BE0FFF763FF08E0FFF778FFF3
S31508001DC005E0FFF787FE02E02020FFF717FE40F246
S31508001DD06413C2F2000393F84230012B02D110209B
S31508001DE0FFF70CFE40F26413C2F20003B3F8441086
S31508001DF00BB2002B0ADD40F26410C2F20000012388
S31508001E0080F84230033009B2FFF760FF08BD00BF13
S31508001E1008B500F051FD08BD10B500F0C9FAB8B113
S31508001E20FEF750FAA0B1FFF793FD00F0D3FA00F0E1
S31508001E30C3FA20F0604020F07F024EF60853CEF237
S31508001E4000031A6000F0B8FA446800F037FDA047AE
S31508001E5010BD00BF70B508E0461C4D1C0B7803701A
S31508001E60FFF7B2FD224630462946531E9CB2002A89
S31508001E70F2D170BD4FF40053C4F2020340F22312AC
S31508001E80C4F267525A6048F6AB12CCF6EF525A6063
S31508001E903422DA60704700BF4FF40053C4F20203DD
S31508001EA01A6942F080021A61704700BF70B506468B
S31508001EB0002442F69015C0F600051BE0FFF784FDE6
S31508001EC004EB440355F82330B34211D804EB44011C
S31508001ED005EB810149680B44B34209D942F69013D0
S31508001EE0C0F6000304EB440203EB8203187A70BDC4
S31508001EF00134E4B20D2CE1D9FF2070BD2DE9F0477D
S31508001F0081460068FFF7D2FFFF284FD0FFF7B2FFE0
S31508001F104FF40053C4F20203DB6813F0010F04D038
S31508001F20FFF7BAFF0020BDE8F0874FF40053C4F26C
S31508001F3002031A6942F001021A6100254FF400549F
S31508001F40C4F2020420E0D9F80080AF0008EB070AC3
S31508001F5009EB07035E68B3B228F8253001E0FFF7FE
S31508001F6033FDE36813F0010FF9D1330CAAF80230F8
S31508001F7001E0FFF729FDE36813F0010FF9D158F8DE
S31508001F800730B34204D101357F2DDCD9012400E0A6
S31508001F9000244FF40053C4F202031A6922F0010226
S31508001FA01A61FFF779FF2046BDE8F0870020BDE8F3
S31508001FB0F08700BF70B50646002442F69015C0F6B5
S31508001FC0000513E0FFF700FD04EB440305EB83036C
S31508001FD01B7AB34208D142F69013C0F6000304EB0D
S31508001FE0440253F8220070BD0134E4B20D2CE9D93D
S31508001FF04FF0FF3070BD00BF70B50646002442F6AC
S315080020009015C0F6000514E0FFF7DEFC04EB440368
S3150800201005EB83031B7AB34209D142F69013C0F647
S31508002020000304EB440203EB8203586870BD0134D5
S31508002030E4B20D2CE8D9002070BD00BFF8B50446FF
S315080020400D4688424CD801284CD90F294CD8FFF7A1
S3150800205011FF4FF40053C4F20203DB6813F0010FBB
S3150800206003D0FFF719FF0020F8BD4FF40053C4F260
S3150800207002031A6942F002021A612046FFF79AFF24
S3150800208006462846FFF796FF04462846FFF7B4FF9C
S315080020902044871BC7F38F2700254FF40054C4F24A
S315080020A002040FE006EB85236361236943F04003CE
S315080020B0236101E0FFF788FCE36813F0010FF9D10B
S315080020C00135ADB2BD42EDD34FF40053C4F202035D
S315080020D01A6922F002021A61FFF7DEFE0120F8BD36
S315080020E00020F8BD0020F8BD0020F8BD08B5C1F3F2
S315080020F0080353B903688B4209D040F8041B4FF410
S315080021000072FFF7A7FE012008BD002008BD0120C8
S3150800211008BD00BF38B504460D4640F2B013C2F2FA
S315080021200003984209D04FF48043C0F60003994251
S3150800213008D0FFF7E3FE48B911E040F2B434C2F222
S31508002140000403E040F2B014C2F200042046294617
S31508002150FFF7CCFF002814BF2046002038BD00201A
S3150800216038BD00BF2DE9F04106460C4617461D4608
S315080021704FEA51284FEA48280368B3F1FF3F03D1D5
S315080021804146FFF7B3FF28B33368434505D03046C9
S315080021904146FFF7BFFF0646F8B13368E41A3444F0
S315080021A0043408F50078FFF70FFC331DE31AB3F57E
S315080021B0007F06D330464146FFF7ACFF064678B1A6
S315080021C0041D17F8013B04F8013B013DEBD1012042
S315080021D0BDE8F0810020BDE8F0810020BDE8F0816F
S315080021E00020BDE8F08100BF40F2B433C2F200031C
S315080021F04FF0FF321A6040F2B013C2F200031A60C1
S31508002200704700BF70B504460D461646FFF74EFEEA
S31508002210FF281BD060190138FFF748FEFF2817D0A2
S31508002220620A4FF48043C0F60003B3EB422F07BFA0
S3150800223040F2B010C2F2000040F2B430C2F2000020
S31508002240214632462B46FFF78DFF70BD002070BD34
S31508002250002070BD70B506460D46FFF727FE0446FA
S3150800226070190138FFF722FE0146FF2818BFFF2C18
S3150800227003D02046FFF7E2FE70BD002070BD00BF08
S3150800228000B583B040F2B013C2F200031B68B3F185
S31508002290FF3F08BF01201CD040F2B013C2F2000372
S315080022A059689A681144DA6811441A6911445A69D6
S315080022B011449A690A44D96953185B4202AA42F83A
S315080022C0043D44F2EC00C0F600000421FFF79AFF33
S315080022D0FFE703B05DF804FB4FF48043C0F6000344
S315080022E0186844F20403C0F600031B68184444F255
S315080022F00803C0F600031B68184444F20C03C0F632
S3150800230000031B68184444F21003C0F600031B6858
S31508002310184444F21403C0F600031B68184444F238
S315080023201803C0F600031A6844F2EC03C0F600036B
S315080023301B6810441844D0F1010038BF00207047CC
S3150800234008B540F2B013C2F200031B68B3F1FF3FB1
S3150800235006D040F2B010C2F20000FFF7CFFD88B1F8
S3150800236040F2B433C2F200031B68B3F1FF3F0BD04F
S3150800237040F2B430C2F20000FFF7C0FD003018BFCB
S31508002380012008BD002008BD012008BD4FF480408B
S31508002390C0F60000704700BF08B5FFF725FF08BD67
S315080023A008B5FFF72FFF08BD08B5FFF753FF08BDAF
S315080023B008B5FFF791FF08BD08B5FFF7E7FF08BDA9
S315080023C008B5FFF75DFF10B1FFF7BAFF08BD00209B
S315080023D008BD00BF4EF21003CEF2000300221A60B9
S315080023E0704700BF08B5FFF7F5FF4EF21003CEF2AF
S315080023F0000341F63F12C0F201025A6000229A60B9
S315080024000521196040F2B853C2F200031A6008BDEC
S315080024104EF21003CEF200031B6813F4803F1FBF71
S3150800242040F2B853C2F200031A68013218BF1A60A4
S31508002430704700BF08B5FFF7EBFF40F2B853C2F28A
S315080024400003186808BD00BF30B400231D460CE021
S31508002450040F092C94BF3034373401F813400001B7
S315080024605C0001340D550133DBB29342F0D330BC26
S31508002470704700BF40F20463C2F2000303F118017B
S31508002480002205E09A745961183318310132D2B224
S31508002490002AF7D09A7400225A6140F20063C2F209
S315080024A0000340F20462C2F200021A60704700BFDD
S315080024B010B440F20063C2F200031B6883B15C6982
S315080024C040F20062C2F20002146019749860D86083
S315080024D000225A741860013908445860987C00E054
S315080024E0FF205DF8044B704738B504460D460128B1
S315080024F007D942F63820C0F600004FF4FC71FFF702
S31508002500B7F940F20463C2F2000304EB440203EB9A
S31508002510C2035A7C1B7C9A4220D040F20463C2F262
S31508002520000304EB440203EBC203DA681570597C16
S3150800253001315974DA680132DA605B689A420FD958
S3150800254040F20463C2F200036200111953F8311015
S31508002550144403EBC403D960012038BD002038BDFC
S31508002560012038BD08B5014640F2F863C2F20003FF
S315080025701878FFF7B9FF08BD38B504460D46012897
S3150800258007D942F63820C0F6000040F21A21FFF7B4
S315080025906FF940F20463C2F2000304EB440203EB52
S315080025A0C2035B7CFBB140F20463C2F2000303EB97
S315080025B0C2039A6812782A70597C013959749A6844
S315080025C001329A605B689A420FD940F20463C2F2FC
S315080025D000036200111953F83110144403EBC403C5
S315080025E09960012038BD002038BD012038BD00BFE4
S315080025F008B5014640F23463C2F200031878FFF7C3
S31508002600BBFF08BD10B50446012807D942F6382095
S31508002610C0F6000040F23A21FFF72AF940F20463B7
S31508002620C2F2000304EB440403EBC403587C10BD58
S3150800263038B5FFF71FFF40F2F864C2F20004601CC9
S315080026404021FFF735FF207040F23465C2F20005DD
S31508002650681C4021FFF72CFF28702378FF2B01D038
S31508002660FF2806D142F63820C0F600007A21FFF787
S31508002670FFF8FEF7BFFB38BD08B50020FDF7F6FDED
S3150800268008BD00BF2DE9F04106460D463F2906D98B
S3150800269042F63820C0F600009921FFF7E9F82846E7
S315080026A0FFF760FF012806D042F63820C0F6000082
S315080026B09D21FFF7DDF8002442F63827C0F600070B
S315080026C04FF0A6080CE0FFF77FF9305DFFF74AFFE9
S315080026D0012803D038464146FFF7CAF80134A4B2A8
S315080026E0A542F0D8BDE8F08110B50446FEF768FFAC
S315080026F040F2FC53C2F200031B78D3B940F2BC5037
S31508002700C2F20000FFF774FF012838D140F2BC532B
S31508002710C2F200031B78A3B340F2FC53C2F20003D3
S3150800272001221A7040F2FD53C2F20003002018700D
S3150800273010BD40F2FD53C2F200031B78144818443A
S31508002740FFF756FF01281ED140F2FD53C2F20003DF
S315080027501A780132D2B21A7040F2BC53C2F20003A0
S315080027601B789A4211D120460949FFF773FB40F2BC
S31508002770FC53C2F2000300221A70012010BD00208B
S3150800278010BD002010BD002010BD002010BD00BFE8
S31508002790BD0500202DE9F04383B040F2F863C2F28C
S315080027A000031878FFF72EFF0546A0B3402D28BF73
S315080027B04025002440F2F867C2F2000742F638289E
S315080027C0C0F6000840F2491940F2B866C2F200069F
S315080027D00FE038780DF10701FFF7CEFE012803D088
S315080027E040464946FFF744F89DF80730335501340B
S315080027F0E4B2AC42EDD340F2B860C2F200004FF446
S3150800280080712A46FEF786FC01202946FEF798FDC8
S315080028100120FEF7F3FC03B0BDE8F0832DE9F84389
S31508002820012040F27861C2F20001FEF7EBFD87B2A3
S31508002830002440F23466C2F2000640F27865C2F21D
S31508002840000542F63828C0F600084FF4B7790BE0C1
S315080028503078295DFFF748FE012803D040464946EF
S31508002860FFF706F80134A4B2BC42F1D30120FEF703
S31508002870D7FCBDE8F88300BF38B54FF2E873C1F658
S31508002880FF731A684FF2EC73C1F6FF731C684FF2B8
S31508002890F073C1F6FF731B68D0180AD0054D294698
S315080028A00822FFF7D1FD204605F110010422FFF7A3
S315080028B0CBFD38BD0200002072B6704762B670477D
S315080028C0F8B500BFF8BC08BC9E467047F8B500BF0F
S315080028D0F8BC08BC9E4670476D61696E2E630000A1
S315080028E01201100100000040501DAC6000010102F9
S315080028F003010000040309042603570069006E005B
S315080029005500530042002000420075006C006B0021
S315080029102000440065007600690063006500000039
S3150800292009022000010100C0320904000002FF006C
S315080029300004070581024000000705010240000067
S315080029401A034F00700065006E0042004C005400E8
S315080029502000550073006500720000002C03570024
S3150800296069006E00550053004200200042007500C1
S315080029706C006B00200049006E0074006500720050
S3150800298066006100630065004F70656E424C540036
S315080029900040000800200000020000000060000857
S315080029A0002000000300000000800008002000004E
S315080029B00400000000A00008002000000500000038
S315080029C000C00008002000000600000000E0000823
S315080029D00020000007000000000001080020000099
S315080029E0080000000020010800200000090000007F
S315080029F000400108002000000A00000000600108ED
S31508002A00002000000B0000000080010800200000E4
S31508002A100C00000000A00108002000000D000000C6
S31508002A2000C00108002000000E00000000E00108B8
S31508002A30002000000F0000002E2E2F2E2E2F2E2EE7
S31508002A402F536F757263652F41524D434D335F5354
S31508002A50544D333246312F7573622E6300000000E1
S30908002A600000000064
S31508002A641C03530045005200310032003300340081
S31508002A74350036003700380039003000991500084B
S31508002A84F10D0008F10D0008F10D0008F10D00081C
S31508002A94F10D0008F10D0008A1150008F10D000854
S31508002AA4F10D0008F10D0008F10D0008F10D0008FC
S31508002AB4F10D000820290008200000000917000865
S31508002AC43117000895160008991600089D1600087F
S31508002AD4F5160008F9160008E5170008F5170008A2
S31508002AE4051800080000000040000000F10D000869
S31508002AF469160008F10D0008F10D0008F10D00082B
S31508002B04F10D0008F10D0008F10D000885160008FE
S31508002B143229000809000000E02800081200000015
S31508002B24F428000804000000402900081A000000E0
S31508002B34F828000826000000000000201C000000F9
S31508002B445C2900082C0000000301000004000000B2
S30D08002B5475010008450100089F
S70508000000F2
